:1002320012010001DC0000107104880800010000B6
:10024200000109022E0001010060010904000004FE
:10025200DCA0B0000705810310000A0705010310A6
:10026200000A0705820240000A0705020240000A4E
:04002000120D0E228D
:10002400E524541FF54E7023AF13EFC4540F54014D
:10003400FFBF0105754C038003754C01E4F54D7B4E
:10004400047A00794C7D02120D9122E54EB401111F
:10005400E4F54CF54D7B047A00794C7D02120D9148
:1000640022E54E6402703EE5295403F54BE5293040
:10007400E70DE54B25E004FF12035B8F4F800AE593
:100084004B25E0FF12035B8F4FE54F30E105754CC4
:10009400018003E4F54CE4F54D7B047A00794C7D52
:0800A40002120D9122120D0E53
:0100AC002231
:1000AD00E524541FF54C701FE52764014526701794
:1000BD00C2AFAF13EF54EFF513D2AF7B007A0079D7
:1000CD0000E4FD120D9122E54C64027034E52745E4
:1000DD0026702EE5295403F54BE52930E70DE54B48
:1000ED0025E004FFE4FD1203BA800AE54B25E0FF8D
:1000FD00E4FD1203BA7B007A007900E4FD120D9144
:04010D0022120D0E9F
:0101110022CB
:10011200E524541FF54C701FE5276401452670172E
:10012200C2AFAF13EF4410F513D2AF7B007A007960
:1001320000E4FD120D9122E54C64027034E527457E
:1001420026702EE5295403F54BE52930E70DE54BE2
:1001520025E004FF7D011203BA800AE54B25E0FF8A
:100162007D011203BA7B007A007900E4FD120D9141
:0401720022120D0E3A
:010176002266
:10017700E527547FFF7D011202727B007A00790028
:06018700E4FD120D9122BF
:10018D00E526F54BE54BB4010C7E027F327D127CEA
:10019D0000120D9F22E54BB4020C7E027F447D2E92
:0901AD007C00120D9F22120D0EC0
:0101B6002226
:1001B700AF14EF5401F54B7B047A00794B7D0112A4
:0201C7000D9198
:0101C9002213
:1001CA00E52745267016FBFAF9FD120D91C2AFAF6D
:1001DA0014EF54FEF514D2AF120D8522E5276401FF
:1001EA0045267019FBFAF9FD120D91120D85120DB3
:1001FA008BC2AFAF14EF4401F514D2AF22120D0E29
:01020A0022D1
:0E020B00E4F54B7B047A00794B7D01120D91D6
:0102190022C2
:10021A00E5274526700EE52945287008FBFAF9FD01
:08022A00120D9122120D0E22AB
:100272008F4B8D4CAF13EFC413540720E002C2AF73
:100282007F037DD0120604E54C6003434B807F025E
:10029200AD4B120604AF13EFC413540720E002D291
:0202A200AF2289
:1002A4008F4CAF13EFC413540720E002C2AF7F0397
:1002B4007DD8120604E54C60097F027D0112060414
:1002C40080077F02E4FD120604AF13EFC413540742
:0602D40020E002D2AF227F
:1002DA008F4B8D4CAF13EFC413540720E002C2AF0B
:1002EA007F037DF31206047F02AD4B1206047F02E0
:1002FA00AD4C120604AF13EFC413540720E002D228
:02030A00AF2220
:10030C008F4BAF13EFC413540720E002C2AF7F032F
:10031C007DFB1206047F02AD4B120604AF13EFC433
:09032C0013540720E002D2AF22B5
:100335007F037DF41206047F021206168F3D7F02AD
:10034500120616AD077C00ED7D00FCED253DFDE4B4
:050355003CFCFEAF05B9
:01035A002280
:02035B00AD07EC
:10035D00AF13EFC413540720E002C2AF7F031206A0
:10036D00047F02120616AE13EEC413540720E002EA
:02037D00D2AFFD
:01037F00225B
:10038000AE077F03EE2440FD1206047F021206161C
:01039000224A
:02039100AE07B5
:10039300AF13EFC413540720E002C2AF7F03EE2470
:1003A30080FD1206047F02120616AE13EEC4135428
:0603B3000720E002D2AFBA
:0103B9002221
:1003BA008D50AE07AF13EFC413540720E002C2AF4B
:1003CA007F03EE2440FD1206047F02AD501206049C
:0D03DA00AF13EFC413540720E002D2AF228E
:0803E7007F037DF612060422DB
:1003EF00AF13EFC413540720E002C2AF7F037DF5B4
:1003FF001206047F021206167508008F097F02127B
:10040F000616EFFEE42509F509EE3508F508AF13DA
:0E041F00EFC413540720E002D2AFAE08AF09BD
:01042D0022AC
:10042E00AF13EFC413540720E002C2AF7F057DFD6A
:10043E001206047F04120616750A008F0B7F041233
:10044E000616EFFEE4250BF50BEE350AF50AAF1393
:0E045E00EFC413540720E002D2AFAE0AAF0B7A
:01046C00226D
:08046D008B3E8A3F8940AD0778
:10047500AF13EFC413540720E002C2AF7F03120687
:10048500047F02120616EF20E00FAF13EFC41354DA
:100495000720E002D2AF7F00227F037DF012060421
:1004A5007F021206168F437F021206168F43E5431D
:1004B500D395414003854143E4F542E542C3954365
:1004C50050197F02120616AB3EAA3FA9408542820B
:1004D500758300EF121835054280E07F037DF21227
:1004E5000604AF13EFC413540720E002D2AFAF43A5
:0104F50022E4
:0604F6008B0C8A0D890E3B
:1004FC00E4F511751201AF13EFC413540720E00299
:10050C00C2AF7512027F037D041206047F0212062D
:10051C0016EF30E04C7F037DF01206047F021206CA
:10052C00168F107F021206168F10E4F50FE50FC31D
:10053C009510501D7F02120616AB0CAA0DA90EE5E4
:10054C000F2511F582E433F583EF121835050F8072
:10055C00DCE5102511F5117F037DF2120604D5128E
:0F056C00A4AF13EFC413540720E002D2AFAF11B6
:01057B00225D
:08057C008B518A528953AD072F
:10058400AF13EFC413540720E002C2AF7F03120677
:10059400047F021206167F037DF01206047F02E434
:1005A400FD1206047F02AD54120604E4F555E55528
:1005B400C3955450197F02AB51AA52A95385558251
:1005C400758300121806FD120604055580E07F03AA
:1005D4007DFA120604AF13EFC413540720E002D2CD
:0305E400AFAF5462
:0105E70022F1
:1005E8008F3D7F03AD3D1206047F037DF1120604A3
:0C05F800E53D70077F037DF2120604222F
:1006E100657070417772697465203D2030782562AC
:1006F100782E0A0043504C4420636F756E74657206
:100701002072656164206261636B203D2030782531
:0C07110062782C2030782562782E0A00D7
:10060400D2A1E42FFFE434FFFE8F82F583EDF0C224
:01061400A144
:0106150022C2
:10061600D2A1E42FFFE434FFFE8F82F583E0FFC210
:01062600A132
:0106270022B0
:100628008F4AD2A1AF14EFC31330E00C7B057A06D2
:1006380079E1854A4F121A04E54A4480F580C29050
:10064800D291D292C292D292E54A547FF580C29258
:05065800D292C2A122B4
:10065D008D4AAB07AA06D2A1E4FFEBFD120604EA10
:10066D00FD7F01120604AF14EFC31330E019E4FF50
:10067D00120616AD077F011206168F508D4F7B05A2
:10068D007A0679F5121A04E54A30E006C2A4D29032
:09069D008004D2A4C290C2A12283
:1006A6008B478A488949900002121806FF33333374
:1006B60054F8FD121859E5F0C41354072DFF12061D
:1006C60028AB47AA48A949900003121886FFAEF046
:0B06D600900005121806FD12065D22C0
:10094F0052656164205265676973746572733A20EA
:10095F004F6666736574203D20307825782C204CC7
:10096F00656E677468203D20307825782C20496E9D
:10097F00646578203D20307825782E0A00577269FB
:10098F007465205265676973746572733A204F6698
:10099F0066736574203D20307825782C204C656E69
:1009AF00677468203D20307825782C20496E646567
:1009BF0078203D20307825782E0A00446174613A02
:0C09CF00200030782562782C20000A00FF
:0609DB000185000184000B
:0E071D00754C217B047A00794C7D01120D9100
:01072B0022AB
:10072C00E52745267013E52B6401452A700B7B01E8
:10073C007A0079857D01120D91E5276401452670BB
:10074C0014E52B6401452A700C7B017A0079847DB9
:10075C0001120D9122E527640245267014E52B64E5
:10076C0004452A700C7B017A0079807D04120D916E
:05077C0022120D0E2207
:10078100E527640145267014E52B6401452A700CA8
:100791007884A633FBFAF9FD120D9122E527640254
:1007A1004526702BE52B6404452A7023AE2AAF2B16
:1007B10078807C007D017B047A0079331217D4782C
:1007C1008576017B007A007900E4FD120D9122E526
:1007D10027640645267013E52B6401452A700B78C2
:0E07E10085F6FBFAF9FD120D9122120D0E2283
:1007EF00AE2AAF2B74862527F974003526A801FC95
:1007FF007D017B047A0079331217D47889E6FC08DF
:10080F00E6FDECFBAF05EF18F6EB08F67886E6FC95
:10081F0008E6FDECFBAF05EF18F6EB08F6D3788A88
:10082F00E6940018E694404004120D0E22AF14EF28
:10083F00C41354075403701FC2AFAF14EF13131335
:10084F00541FFEEF54E7FFEE045403FE33333354CB
:10085F00F84FF514D2AF22C2AFAF14EF549F4440FC
:04086F00F514D2AFFB
:010873002262
:10087400E52430E751AF14EFC31330E01B7B057A56
:1008840009794F85264F852750852A51852B528516
:100894002853852954121A04E529B47217E528B49B
:1008A4000412E5274526700CE52B6401452A7004E3
:1008B40012071D22E529B47309E528B404041207BC
:1008C4002C22120D0E22AF14EFC31330E04F7B0520
:1008D4007A09798C85264F852750852A51852B5294
:1008E400852853852954121A047B057A0979CA127A
:1008F4001A04E4F54BC3E54B952BE4952A50157B7C
:10090400057A0979D17433254BF8E6F54F121A04A8
:10091400054B80E17B057A0979D9121A04E529B4DB
:100924007117E528B40412E5274526700CE52B64FD
:1009340006452A70041207EF22E529B47309E52855
:0A094400B4040412078122120D0E04
:01094E002286
:100EEF00486F73745F746F5F646576696365004400
:100EFF0065766963655F746F5F686F7374004465CF
:100F0F007669636500496E74657266616365004555
:100F1F006E64706F696E74283029004F7468657243
:100F2F00005374616E6461726400436C617373008B
:100F3F0056656E646F7200526573657276656400F4
:100F4F004745545F53544154555300434C45415208
:100F5F005F464541545552450052455345525645FB
:100F6F0044005345545F4645415455524500524540
:100F7F00534552564544005345545F4144445245EE
:100F8F005353004745545F44455343524950544FC0
:100F9F0052005345545F44455343524950544F52A6
:100FAF00004745545F434F4E4649475552415449B8
:100FBF004F4E005345545F434F4E4649475552419C
:100FCF0054494F4E004745545F494E544552464190
:100FDF004345005345545F494E544552464143459E
:100FEF000053594E435F4652414D4500526571754E
:100FFF006573742054797065203D2025732C205221
:10100F00657175657374203D2025732E0A00526536
:10101F0071756573742054797065203D2025732C8C
:10102F00206252657175657374203D20307825629A
:10103F00782E0A000A5044495553424431322065F4
:10104F0076616C756174696F6E20626F6172642076
:10105F006669726D776172652056322E332E0A00E3
:10106F00436F70797269676874202863292050680C
:10107F00696C6970732053656D69636F6E64756316
:10108F00746F72732C20313939392E0A0052652D45
:10109F00636F6E6E656374205044495553424431FB
:1010AF0032206576616C756174696F6E20626F6155
:1010BF00726420746F205553422E0A00436F6E7472
:1010CF00726F6C207374617465203D205553425FBD
:1010DF0049444C452E00436F6E74726F6C207374CD
:1010EF00617465203D205553425F52454345495633
:1010FF00452E00436F6E74726F6C2073746174654C
:10110F00203D205553425F5452414E534D49542E6A
:10111F000020436F6E74726F6C446174612E77435D
:10112F006F756E74203D2025782E0A00456E647011
:10113F006F696E742034202842756C6B204F757464
:10114F002920537461747573203D202562782C20FB
:10115F00456E64706F696E742035202842756C6B14
:10116F0020496E2920537461747573203D202562C8
:10117F00782E0A00444D415F5374617465203D2001
:10118F00444D415F49444C452E0A00444D415F5345
:10119F0074617465203D20444D415F52554E4E4958
:1011AF004E472E0A00444D415F5374617465203DD4
:1011BF0020444D415F50454E44494E472E0A00434F
:1011CF00504C4420636F756E746572207265616454
:1011DF00206261636B203D2030782562782C2030AF
:1011EF00782562782E0A004C617374204465766905
:1011FF00636520526571756573743A20626D52652F
:10120F00717565737454797065203D20307825624F
:10121F00782C2062526571756573743D2030782586
:10122F0062782C207756616C7565203D20307825CB
:10123F00782C20774C656E677468203D20307825B8
:10124F00782C2077496E646578203D20307825789A
:10125F002E0A00446174613A200030782562782CA0
:10126F0020000A00566572626F7365204D6F6465CA
:10127F00203D204F4E2E0A00566572626F73652017
:10128F004D6F6465203D204F46462E0A0042757310
:10129F00207265736574210A0053757370656E64EF
:1012AF00206368616E6765210A0057616974206663
:1012BF006F722031207365636F6E64202E2E2E0A9D
:1012CF00000500240500AD050020050112050020D2
:1012DF0005017705018D0500200501B70501CA0538
:1012EF00020B05021A05002005002005002005004D
:1012FF002005002005002005002005002005002006
:10130F000500200500200500200500200500200510
:10131F0000200500200508740500200500200500A9
:10132F0020050EEF050EFE050F0D050F14050F1E00
:10133F00050F2A050F30050F39050F3F050F46051D
:10134F000F4F050F5A050F68050F71050F7D050F1C
:10135F0086050F92050FA1050FB0050FC2050FD41B
:06136F00050FE2050FF07E
:0309E10001230FE0
:1009EB008F498D4AE549C4135407F5497048E549C9
:1009FB0075F003A42442F582E43413F583E493FBEE
:100A0B00740193FA7402938B4F8A50F551E54A7532
:100A1B00F003A4244EF582E43413F583E493FB74C2
:100A2B000193FA7402938B528A53F5547B057A0F18
:100A3B0079FB121A0422AF14EFC31330E02BE549F4
:100A4B0075F003A42442F582E43413F583E493FB9D
:100A5B00740193FA7402938B4F8A50F551854A5265
:0A0A6B007B057A10791D121A04228F
:100A75005389F0438901E4F58AF58CD2A9D28CD249
:040A8500B9D2AF2211
:070A8900C288D2A8C2B82206
:0A0A90007580FF7590FF75A0FF222E
:100A9A00759852438780758920758869758DF32208
:010AAA002229
:100AAB00754501120A90120A9A120A75120A897B6D
:100ABB00057A107943121A047B057A10796F121A92
:100ACB00047B057A10799C121A04120D3BE54570D4
:100ADB0003020D09AF13EF30E014C2AFAF13EF54A5
:100AEB00FEF513D2AFAF14EF30E003120E162098C1
:100AFB0003020C80121CF4EF24F37003020C492444
:100B0B00A4601424F37003020C4E24046003020C43
:100B1B00801203E7020C80AF13EFC413135403547A
:100B2B0003700B7B057A1079CB121A048030AF134C
:100B3B00EFC4131354035403FFBF020B7B057A104E
:100B4B0079E5121A048017AF13EFC413135403542F
:100B5B0003FFBF01097B057A117902121A047B0589
:100B6B007A117920852E4F852F50121A047F04128B
:100B7B000391C0077F051203918F50D04F7B057AED
:100B8B0011793B121A04AF14EFC4135407540370BA
:100B9B000B7B057A117983121A04802EAF14EFC4E4
:100BAB001354075403FFBF010B7B057A11799A127B
:100BBB001A048016AF14EFC41354075403FFBF027B
:100BCB00097B057A1179B4121A04D2A1E4FF12063B
:100BDB0016C0077F011206168F50D04F7B057A1176
:100BEB0079CE121A04C2A17B057A1179F685244FAE
:100BFB00852550852651852752852A53852B54856B
:100C0B002855852956121A047B057A127962121A15
:100C1B0004E4F546C3E546952BE4952A50157B0570
:100C2B007A12796974332546F8E6F54F121A0405E2
:100C3B004680E17B057A127971121A048037120D06
:100C4B003B8032AF14EFC31320E0167B057A127989
:100C5B0073121A04C2AFAF14EF4402F514D2AF8073
:100C6B00147B057A127987121A04C2AFAF14EF54B2
:100C7B00FDF514D2AFAF13EFC31330E014C2AFAF17
:100C8B0013EF54FDF513D2AF7B057A12799C121A30
:100C9B0004AF13EF1313543F30E017C2AFAF13EF92
:100CAB0054FBF513D2AF120D0D7B057A1279A812F6
:100CBB001A04AF13EF131313541F30E00EC2AFAF70
:100CCB0013EF54F7F513D2AF120E96AF14EF1313B5
:100CDB0013541F54037003020AD8C2AFAF14EF139F
:100CEB001313541FFEEF54E7FFEE145403FE33337C
:100CFB003354F84FF514D2AF120E5C020AD8120A15
:010D0B00AA3D
:010D0C0022C4
:010D0D0022C3
:0F0D0E00E4FF7D011203BA7F017D011203BA22B7
:080D1D007F067D431202DA2279
:100D2500C2AFE4F513F514D2AF7FC012030C7F16E2
:060D35007D431202DA22E8
:100D3B00C2B4C2B5120D1D7B057A1279B9121A0411
:100D4B0085184A8517498516488515477F147E00F7
:100D5B007D007C001218F8AF4AAE49AD48AC471283
:100D6B0018C01218F8AF18AE17AD16AC151218D371
:090D7B0040DA120D25D2B4D2B504
:010D8400224C
:050D8500E4FF1202A4CE
:010D8A002246
:060D8B007F011202A42208
:0E0D9100EDD3941050077F018D5412057C2283
:100D9F008E4C8F4DE4F52EF52FD3E52D9DE52C9C34
:100DAF0040048C2C8D2D753005854C31854D32C30B
:100DBF00E52D9410E52C940040277F01AB30AA312C
:100DCF00A93275541012057C7410252FF52FE435B8
:100DDF002EF52EC2AFAF13EF543F4440F513D2AFF1
:100DEF00227F01AA4CA94D7B05852D5412057CE568
:100DFF002D252FF52FE52C352EF52EC2AFAF13EF86
:070E0F00543FF513D2AF229E
:100E1600A2A682A5E433F52253220FE522652360BC
:100E26000E7F037B047A00792275540112057C85B6
:100E36002223AF14EF1313543F30E019C2AFAF149F
:100E4600EF54FBF514D2AF788FE6FF13B392B4EFED
:050E5600A2E1B392B51A
:010E5B002274
:100E5C00AF14EF547FF5147B017A0079861206A645
:100E6C00C2AFAF14EF549F4420F514D2AF7B007A7D
:100E7C00007900E4FD120D91788BE630E0067F0CD2
:0A0E8C0012030C227F0412030C2253
:100E9600E5245460F547E525540FF548AF47FD12A4
:100EA60009EBE547701DE54875F003A424D0F582EB
:100EB600E43412F583E493740193FA740293F912FD
:100EC600193722E547B4401DE54875F003A4240010
:100ED600F582E43413F583E493740193FA74029370
:080EE600F912193722120D0E5A
:010EEE0022E1
:0609E400041500000000F4
:03000B0002137568
:10137500C0E0C0F0C083C082C0D0C000C004C005BA
:10138500C006C007C2AFAF18AE17AD16AC15121820
:10139500F87F017E007D007C001218C08F188E1723
:1013A5008D168C15AF13EF4401F513D2AFD007D0CE
:1013B50006D005D004D000D0D0D082D083D0F0D0D4
:0213C500E03214
:030003000213C71E
:1013C700C0E0C0F0C083C082C0D0C000C001C0026E
:1013D700C003C004C005C006C007C2AF121403D2C1
:1013E700AFD007D006D005D004D003D002D001D0AB
:0C13F70000D0D0D082D083D0F0D0E03203
:10140300AF13EF4420F5131203358E3B8F3CE53CBD
:10141300453B6055E53C30E60C121474AF13EF44C2
:1014230002F5138044E53B30E003121622E53C301D
:10143300E707AF13EF4404F513E53C30E10312155E
:1014430086E53C30E003121475E53C30E3031216E5
:1014530052E53C30E203121658E53C30E503121620
:1014630076E53C30E40312167CAF13EF54DFF5133B
:011473002256
:011474002255
:10147500E4FF120380EF20E503021539E4F52CF5AE
:101485002DF52EF52FFF7B047A007924754108127E
:10149500046DEF64086016E4FF7D011203BA7F0155
:1014A5007D011203BAAF13EF543FF51322E526FD74
:1014B500E527F526EDF527E528FDE529F528EDF5E0
:1014C50029E52AFDE52BF52AEDF52BE4FF1205E8C4
:1014D5007F011205E8852A2C852B2DE4F52EF52FA5
:1014E500E52430E70FAF13EF4408F513AF13EF54BE
:1014F5003FF51322E52B452A700FAF13EF4408F58E
:1015050013AF13EF543FF51322D3E52B9408E52AC7
:1015150094004016AF13EF543FF513E4FF7D01121D
:1015250003BA7F017D011203BA22AF13EF543F4482
:1015350080F51322AF13EFC413135403540364024D
:101545007037FF7433252FF9E4FA7B0475411012C7
:10155500046DEF252FF52FE4352EF52EBF100BC3A7
:10156500E52F952DE52E952C4016AF13EF4408F584
:1015750013AF13EF543FF51322AF13EF543FF51399
:011585002243
:10158600C3E52D952FF53EE52C952EF53D7F0112F1
:101596000380AF13EFC41313540354036401707B29
:1015A600C3E53E9410E53D6480948040297F01ABFD
:1015B60030E532252FF9E531352EFA75541012052E
:1015C6007C7410252FF52FE4352EF52EAF13EF542E
:1015D6003F4440F51322E53E453D60287F01AB3090
:1015E600E532252FF9E531352EFA853E5412057C74
:1015F600E53E252FF52FE53D352EF52EAF13EF549D
:101606003FF51322E53E453D70117F01FBFAF9F5E2
:0B1616005412057CAF13EF543FF51396
:0116210022A6
:10162200AF14EFC41354075403FFBF021BAF14EFF0
:10163200131313541FFEEF54E7FFEE045403FE335B
:10164200333354F84FF51422AF14EF549FF514229C
:061652007F031203802259
:101658007F021203807F027B017A00798C7541102A
:0D16680012046DEF6007AF14EF4404F51499
:011675002252
:061676007F051203802233
:06167C007F04120380222E
:0300000002168263
:0C168200787FE4F6D8FD75819B0216C944
:10170E00E709F608DFFA8046E709F208DFFA803EBD
:10171E0088828C83E709F0A3DFFA8076E309F60866
:10172E00DFFA806EE309F208DFFA806688828C8326
:10173E00E309F0A3DFFA805A89828A83E0A3F608D0
:10174E00DFFA804E89828A83E0A3F208DFFA8042B4
:10175E0080AE80B480BA80C480CA80D080DA80E443
:10176E0080378023805389828A83ECFAE493A3C85E
:10177E00C582C8CCC583CCF0A3C8C582C8CCC583EE
:10178E00CCDFE9DEE7800D89828A83E493A3F60835
:10179E00DFF9ECFAA9F0EDFB2289828A83ECFAE0FC
:1017AE00A3C8C582C8CCC583CCF0A3C8C582C8CC9B
:1017BE00C583CCDFEADEE880DB89828A83E493A3EB
:1017CE00F208DFF980CC88F0ED14B4040050C32485
:1017DE001E83F582EB14B4050050B72415832582C1
:1017EE00F582EF4E60ACEF60010EE58290175E73EE
:0817FE00000402000C060012B9
:10180600BB020CE58229F582E5833AF583E02240A6
:1018160003BB0406E92582F8E622400DE58229F598
:0F18260082E5833AF583E49322E92582F8E222F2
:10183500F8BB020DE58229F582E5833AF583E8F0E8
:10184500224003BB0406E92582C8F6225005E92596
:0418550082C8F22231
:10185900BB020A89828A83E0F5F0A3E0224003BB38
:10186900040687F009E71922400C89828A83E493E8
:0D187900F5F074019322E3F5F009E3192264
:10188600BB0210E58229F582E5833AF583E0F5F09F
:10189600A3E0224003BB0409E92582F886F008E6A6
:1018A60022400DE5832AF583E993F5F0A3E9932217
:0A18B600E92582F8E2F5F008E222CD
:1018C000EF251CFFEE351BFEED351AFDEC3519FC3E
:0318D00002191FDB
:1018D300C3EF951CF8EE951B48F8ED951A48F8EC04
:1018E300951948F892D5D082D083121917E8A2D55A
:0518F300C083C0822249
:1018F800E51D051D6010D0F0D0E0C019C01AC01B4E
:10190800C01CC0E0C0F08F1C8E1B8D1A8C1922AF32
:101918001CAE1BAD1AAC19E51D146010D0F0D0E058
:0F192800D01CD01BD01AD019C0E0C0F0151D2262
:061937008A838982E4733B
:1019A200E55B244FF8E6055B22784C300702784F5E
:1019B200E475F00112196C02193D2000EB7F2ED262
:1019C200008018EF540F2490D43440D4FF30040B1D
:1019D200EF24BFB41A0050032461FFE55C600215D6
:1019E2005C055FE55F7002055E30070D784CE475BB
:1019F200F00112196CEF021958021CFE7403D2078F
:101A02008003E4C207F55B8B4C8A4D894EE4F55C9A
:101A1200F55EF55FE55C60077F201219DD80F5F564
:101A22005DC201C200C202C203C205C206C20812DE
:101A320019ABFF700D3007057F001219EEAF5FAED4
:101A42005E22B42561C2D5C2041219ABFF24D0B400
:101A52000A00501C75F00A20D50DC55CA4255CF562
:101A62005C7002D20380E0C55DA4255DF55D80D780
:101A720024CFB41A00EF5004C2E5D204021BE7D20D
:101A82000180C2D20080BED20280BAD2D580B8D242
:101A92000580B27F201219DD2002077401B55C00B7
:101AA20040F11219A2FF1219DD021A16D208D2064B
:101AB20080931219A2FB1219A2FA1219A2F94A4B27
:101AC200700679B37A1C7B05200233E55C602FAF88
:101AD2005DBF00011F7E008E8275830012180660B2
:101AE200050EEE6F70F1C2D5EBC0E0EAC0E0E9C0CE
:101AF200E0EE121C2BD0E0F9D0E0FAD0E0FB121994
:101B02003DFF60A5EBC0E0EAC0E0E9C0E01219DDEC
:101B1200D0E02401F9D0E03400FAD0E0FBE55D60CA
:101B2200DDD55DDA80837B057A1C7927D202809825
:101B3200791080027908C206C2088008D2D5790AD3
:101B42008004790AC2D5E4FAFDFEFF1219A2FC7BD9
:101B5200082001131219A2FD7B1030000A1219A2EB
:101B6200FE1219A2FF7B20EC3382D592D55013C30B
:101B7200E43000069FFFE49EFEE42001039DFDE4A5
:101B82009CFCE4CBF8C201EC700CCFCECDCCE824A7
:101B9200F8F870F38017C3EF33FFEE33FEED33FD39
:101BA200EC33FCEB33FB994002FB0FD8E9EB30013D
:101BB20005F8D0E0C448B201C0E00AEC4D4E4F78BF
:101BC200207B0070C2EAC0E0121C2DD0F0D0E020D1
:101BD2000104C4C0E0C4B201C0F01219C6D0F0D5ED
:101BE200F0EB021A1612197C1AB4531B32581A85DA
:101BF2004C1A81421B364F1B3E441B3E491A9A43E4
:101C02001B44551B28461B28451B28471CD7501A26
:101C1200892D1A8D2E1AB02B1A91231AAE201CC2AE
:101C22002A00001AA83F3F3F00790AA2D5200314D8
:101C3200300509B910020404B9080104A2D520062E
:091C420002500104200266920226
:101C4B00B55C005032C0E07F203003177F30A2021A
:101C5B0072067205500D121C82C202C206C2057FAB
:101C6B0030800F300503E9C0E01219DD300503D0D9
:101C7B00E0F9D0E0B55CCE3005177F30B9100C120F
:101C8B0019DD7F583004077F788003B908031219D8
:101C9B00DD3002057F2D0219DD7F202008F87F2B18
:101CAB002006F322920280CF286E756C6C29002DD2
:101CBB004958504443D2011219A23001F8C201789D
:101CCB005C30D504D200785DF6021A471219A2B423
:101CDB0006004001E4901CBA931219CE743A121903
:091CEB00CED203755C04021B3229
:0A1CF4003098FDAF99C2987E0022DF
:10168E00020AABE493A3F8E493A34003F68001F2BD
:10169E0008DFF48029E493A3F85407240CC8C3335D
:1016AE00C4540F4420C8834004F456800146F6DF2C
:1016BE00E4800B01020408102040809009DBE47ED8
:1016CE00019360BCA3FF543F30E509541FFEE49321
:1016DE00A360010ECF54C025E060A840B8E493A3E8
:1016EE00FAE493A3F8E493A3C8C582C8CAC583CA13
:1016FE00F0A3C8C582C8CAC583CADFE9DEE780BECB
:0109EA00000C
:10193D00BB020689828A83E0224003BB0402E722B0
:0B194D00400789828A83E49322E32292
:10195800BB020689828A83F0224003BB0402F72275
:041968005001F32215
:10196C00FAE6FB0808E6F925F0F618E6CA3AF6227C
:10197C00D083D082F8E4937012740193700DA3A3FA
:10198C0093F8740193F5828883E47374029368600E
:06199C00EFA3A3A380DF0E
:101CFE00EFB40A07740D121D09740A309811A899D1
:101D0E00B8130CC2983098FDA899C298B811F63045
:071D1E0099FDC299F599221D
:00000001FF
